:100000001DC037C036C035C034C033C032C031C067
:1000100030C02FC02EC02DC02CC02BC02AC029C07C
:1000200028C027C026C025C024C05DC1DCC021C0B7
:1000300020C01FC01EC01DC0B3C01BC011241FBEE6
:10004000CFEFD1E0DEBFCDBF11E0A0E0B1E0E2E64E
:10005000FAE002C005900D92AE31B107D9F721E068
:10006000AEE1B1E001C01D92AB39B207E1F700D4B7
:10007000F6C4C6CFCF93DF93EC0109900020E9F7D7
:100080002197C81BD90BCF30D10514F0CEE0D0E0BA
:10009000AE01BC0186E291E0C3D4FE01EA5DFE4FF1
:1000A0001082C0932501DF91CF910895809138018E
:1000B0008730C0F4833020F0E5EEFFE0E49105C026
:1000C000E7EEFFE0E491823019F48350823010F4BF
:1000D00081E001C080E0E093740098ED909371009E
:1000E000809373000895CF93DF931F92CDB7DEB74F
:1000F0008091860087FF10C08091860084FF05C034
:1001000080918000898382E008C08091800089838B
:100110008093690180E001C081E00F90DF91CF9171
:10012000089530911F0120911E013217E1F02091B6
:100130001F0130911E01231B2F71382FFC018E2FC0
:10014000831B821770F4A0911E01B0E0A558BE4F2A
:100150008C91819380911E018F5F8F7180931E011E
:10016000EECF822F089580E008958091960085FF5C
:1001700016C0F8949091210180912001981771F098
:10018000E0912001F0E0E65CFE4F808180939000DA
:10019000809120018F5F8F71809320017894089562
:1001A0001F920F920FB60F9211242F933F934F93EC
:1001B0005F936F937F938F939F93AF93BF93EF93CF
:1001C000FF93D3DFFF91EF91BF91AF919F918F91FB
:1001D0007F916F915F914F913F912F910F900FBE43
:1001E0000F901F9018951F920F920FB60F92112427
:1001F0002F933F938F939F93EF93FF93809186006C
:1002000030918000E091240184FD07C081E08E0FD1
:100210008F7190911E0189130AC080911F018093F4
:10022000240180915A018F5F80935A011AC0209156
:100230002301211106C0932F92959F709F5F909389
:100240002201F0E0E558FE4F30838093240191E0D5
:10025000920F9093230120912201921304C0809366
:100260001F0110922301FF91EF919F918F913F9178
:100270002F910F900FBE0F901F9018951F93CF9343
:10028000DF931F92CDB7DEB7109121011F5F1F7161
:1002900090912001191304C0898367DF8981F8CF09
:1002A000E0912101F0E0E65CFE4F80831093210194
:1002B000F8945BDF78940F90DF91CF911F910895B0
:1002C000CF93DF93D0916A01D295DF70C0E0EC2F1D
:1002D000F0E0E659FE4F8081D1DFCF5FDC17B8F741
:1002E000DF91CF9108951895CF93DF931F92CDB7EB
:1002F000DEB7E0913801E730C8F5F0E0E050FF4F9D
:1003000080819091800099839981998310928600D1
:10031000109285001092840010928300D29810925F
:100320008200382F3F7730938100881F8827881FED
:10033000880F8093860090E99093850026E02093B3
:10034000840010928300909165009E7F90936500D9
:10035000D59A10929200309391008093960088E491
:100360008093950020939400109293000F90DF915A
:10037000CF910895CF93DF93C0E0D0E08CEC9CE167
:100380000197F1F700C00000809138018F5F482F7E
:100390004470682F6270817051D28CEC9CE101979F
:1003A000F1F700C000009FDE8130E9F3823029F4CC
:1003B00040E060E08FEF42D20CC0809169018A304A
:1003C00021F04FEF60E080E039D2809169018A30FE
:1003D00099F0809138018F5F863019F08093380151
:1003E00002C0109238018FEF97E40197F1F700C037
:1003F00000005CDE79DFC0CF81EE92E00197F1F77B
:10040000000040E06FEF80E019D2CD2B19F4C1E07D
:10041000D0E0B4CFDF91CF910895909121018091E8
:100420002001981711F0A1DEF8CF10928500CA992B
:10043000FECF1092900008958230C9F028F48823EE
:1004400041F0813049F008958330D1F0843019F1C2
:100450000895E3DFDFD002C0E0DF4AD186E69EE008
:100460000197F1F7000080E980938500089580915D
:100470003901869590E0855A9E4FD4D089E008C016
:1004800080913901869590E0855A9E4F32D187E060
:100490008093390108955FD0811109C08FE49BE4F6
:1004A000909327018093260182E08093250108958F
:1004B000B89A85E08A95F1F7B99A0895B99885E0D8
:1004C0008A95F1F7B898089598E025E02A95F1F714
:1004D00087FF02C0B89801C0B89A880F25E02A9516
:1004E000F1F7B9982AE02A95F1F7B99A915069F78E
:1004F000B8988AE08A95F1F7B9989AE09A95F1F759
:1005000086B3B99A25E02A95F1F781700895B898D5
:1005100038E020E045E04A95F1F7B9984AE04A957D
:10052000F1F7220FB099216045E04A95F1F7B99AA9
:10053000315081F7892B09F4B89A85E08A95F1F753
:10054000B9984FE04A95F1F7B99A85E08A95F1F7A5
:10055000B898822F0895CF93DF93CBE0D0E088B393
:100560008C7F88BB87B38C7F87BB86E69EE0019734
:10057000F1F700009DDF8AEAA7DF811115C02197FE
:10058000209779F0B89888E090E0B99A2AE02A9507
:10059000F1F7B9982AE02A95F1F701970097A9F7A2
:1005A000DECF82E191E00DC089DF86E69EE0019713
:1005B000F1F700007DDF8AE387DF882331F086E1F1
:1005C00091E058DD7BDFC1E021C080E27DDF8FEB71
:1005D0007BDF74DF9AE09A95F1F76ADF8CE374DFD2
:1005E000C82F882331F08AE191E044DD67DFC2E063
:1005F0000DC080E269DF8CEF67DF80E665DF81E0B8
:1006000063DF82E061DF80E05FDF58DF8C2FDF9106
:10061000CF9108954DDF8CE357DF82E255DF81E013
:1006200053DF4CCF0F931F93CF93DF93EC0140DF49
:100630008CE34ADF88E248DF41DF8AE08A95F1F700
:1006400037DF8DE341DF80E090E061DF082F10E0CD
:10065000102F00271983088380E090E058DF082BD3
:100660001983088380E090E052DF082F10E0102FFC
:1006700000271B830A8380E090E049DF082B1B835F
:100680000A8380E090E043DF082F10E0102F00275E
:100690001D830C8381E090E03ADF082B1D830C83DF
:1006A0000DDF8AE08A95F1F703DF8CE30DDF8EE240
:1006B0000BDF04DF8AE08A95F1F7FADE8DE304DFD1
:1006C00080E090E024DF082F10E0102F00271F8328
:1006D0000E8381E090E01BDF082B1F830E83EEDE8C
:1006E0008AE08A95F1F7DF91CF911F910F910895DC
:1006F00008950F931F93CF93DF93EC01D9DE8AE324
:10070000E3DE88EAE1DEDADE8AE08A95F1F7D0DE20
:100710008BE3DADE80E090E0FADE082F10E0198348
:10072000088380E090E0F3DE182B1983088380E0D3
:1007300090E0EDDE082F10E01B830A8380E090E05C
:10074000E6DE182B1B830A8380E090E0E0DE082FB2
:1007500010E01D830C8381E090E0D9DE182B1D830F
:100760000C83DF91CF911F910F91A8CE1F93CF9350
:10077000DF931F92CDB7DEB7182F698399DE8CE324
:10078000A3DE812FA1DE6981862F9EDE0F90DF918F
:10079000CF911F9193CE1F93CF93DF931F92CDB72D
:1007A000DEB7182F85DE8CE38FDE812F80688CDE2C
:1007B00085DE8AE08A95F1F77BDE8DE385DE81E0D8
:1007C00090E0A5DE89837ADE89810F90DF91CF9159
:1007D0001F9108951F93CF93DF931F92CDB7DEB77C
:1007E000182F698365DE8AE36FDE812F6DDE6981F4
:1007F000862F6ADE0F90DF91CF911F915FCE1F93FE
:10080000CF93DF931F92CDB7DEB7182F51DE8AE367
:100810005BDE812F806858DE51DE8AE08A95F1F731
:1008200047DE8DE351DE81E090E071DE898346DEB4
:1008300089810F90DF91CF911F910895BA9A4F93BC
:100840006F938F9343E05F9168E057FF06C032E0FB
:10085000C29A3A95F1F7C29805C0C29AC29832E09E
:100860003A95F1F7550F6A9581F74A9561F7089522
:10087000F89487E090E0DDD080933801863010F066
:100880001092380113DC30DD75DD8AE0F7DC8AE098
:10089000F5DC6091380187E090E0D3D05CDE811117
:1008A00009C08FE49BE4909327018093260182E0A6
:1008B0008093250141E061E081E0C0DF789400E8A9
:1008C00016E08AE691E02DDC90E00097D1F32091CC
:1008D0006A012F70243009F452C028F4223051F0FC
:1008E000233041F14AC0253009F46BC02B3009F4A4
:1008F0006DC043C0019749F4E3DC4091370160913A
:100900003501809136019ADFDCCF80916B01811136
:100910000DC080916C018093350180916D018093B1
:10092000360180916E0180933701CBCF8150809347
:100930006B0123C0019729F080916B018F5F809339
:100940006B01BEDCC0912501CC2309F4BACF109213
:100950006B01D0E0AE0166E271E08CE691E060D020
:10096000AE014F5F5F4F94E0440F551F9A95E1F73A
:10097000436040936A0110922501A2DCA2CF8091CE
:100980006B018F5F80936B019BDCC0913901CC239D
:1009900009F497CF10926B01D0E0AE016AE571E0E7
:1009A0008CE691E03DD0AE014F5F5F4F84E0440F95
:1009B000551F8A95E1F7446040936A01109239010E
:1009C000DCCF7EDC80916B0137DD7BCF79DC41E0D1
:1009D00060E181E033DF4BE050E066E071E08AE601
:1009E00091E011D0892B09F06CCF8FEF9FE8019730
:1009F000F1F700C00000F89441E061E080E11EDF03
:100A0000F80109955ECFFB01DC0104C08D910190D6
:100A1000801921F441505040C8F7881B990B089564
:100A2000FB01DC0102C001900D9241505040D8F70B
:100A30000895E199FECF1FBA8EBBE09A99278DB336
:100A40000895262FE199FECF1CBA1FBA8EBB2DBB8D
:100A50000FB6F894E29AE19A0FBE01960895F894C1
:020A6000FFCFC6
:100A6200032F00018080AB626F6F746C6F616465ED
:0E0A72007200424552004C4641004D46410084
:00000001FF
